:100000000C9449000C9466000C9466000C946600F5
:100010000C9466000C9466000C9466000C946600C8
:100020000C9466000C9466000C9466000C946600B8
:100030000C9466000C9466000C9466000C949E046C
:100040000C94EA040C944F030C9466000C94660024
:100050000C9466000C9466000C9466000C94660088
:100060000C9466000C9466000C9466000C94660078
:100070000C9466000C9466000C9466000C94660068
:100080000C9466000C9466000C94660000081C1822
:10009000141011241FBECFEFD0E1DEBFCDBF11E0A1
:1000A000A0E0B1E0EEE5FAE000E00BBF02C007908F
:1000B0000D92A030B107D9F711E0A0E0B1E001C086
:1000C0001D92A433B107E1F70C945F030C94000078
:1000D0008FB7F894992708958FBF0895880F949843
:1000E00096E087FF02C0979A01C097989698969AD3
:1000F000880F915097FFF5CF979A9698969A949A71
:1001000097E067FF02C0979A01C097989698969AD1
:10011000660F915097FFF5CF949A979A969A089503
:10012000982FE82FFF27EF5CFE4F80818F3FB9F4B7
:1001300080913301891799F0809130018F3F19F434
:100140009093300107C080913301E82FFF27EF5CC7
:10015000FE4F90839093330181E090E0089580E01A
:1001600090E00895CF93DF938FB7F894682F7727A7
:10017000A0912601B0912701C0912801D0912901B9
:1001800082B706B600FE04C01196C11DD11D82B70C
:10019000282F33274427552788279A2FAB2FBC2F8A
:1001A000822B932BA42BB52B6FBFBC01CD01DF910C
:1001B000CF910895AF92BF92CF92DF92EF92FF92CC
:1001C0000F931F93CF93DF930E94B200FC01EB01CA
:1001D0002091200130912101409122015091230171
:1001E0007B018C01E21AF30A040B150B1092240117
:1001F00080911C0190911D01A0911E01B0911F01E1
:10020000E816F9060A071B07C0F0EE24FF24870151
:10021000280F391F4A1F5B1F2093200130932101B3
:100220004093220150932301E0921C01F0921D01A2
:1002300000931E0110931F0163C05C016D01AE1895
:10024000BF08C00AD10A8601750161E0A61661E007
:10025000B60660E0C60660E0D60690F080E0A8161C
:1002600080E0B80681E0C80680E0D80610F08FEF85
:1002700004C0BB27AD2D9C2D8B2D8093240158C02D
:1002800061E8A616B104C104D10430F1C058DF4FB3
:10029000EF4FFF4FC0932001D0932101E093220143
:1002A000F0932301C058D040E040F04080E89FEF39
:1002B000AFEFBFEFE80EF91E0A1F1B1FE0921C01F3
:1002C000F0921D0100931E0110931F0190E8E92E8A
:1002D000F12C012D112D14C0280F391F4A1F5B1F4F
:1002E0002093200130932101409322015093230158
:1002F00010921C0110921D0110921E0110921F01FC
:100300006E2D82B7282F8C1B8E5F8E1518F0622FF2
:100310006E5F01C06C0F662309F461E0615000B6A6
:1003200001FCFDCF61BF82E086BF87B7826087BFD7
:10033000DF91CF911F910F91FF90EF90DF90CF90C1
:10034000BF90AF9008956F927F928F929F92AF92DD
:10035000BF92CF92DF92EF92FF920F931F93CF93B2
:10036000DF935B016C0110E0EE24FF2460E071E09C
:10037000FB01008501FF49C0208131814281538109
:10038000D601C501821B930BA40BB50B648075804D
:100390008680978086159705A805B905B0F100FFFE
:1003A00003C00D7F008709C0260D371D481D591D4C
:1003B000FB012083318342835383F1E0EF16F10484
:1003C000A1F082E0E816F10424F4E114F10431F024
:1003D0001CC0E2E0EE16F10479F017C08FB7F89474
:1003E000282F33278BB394E00DC08FB7F894282FB4
:1003F00033278BB392E006C08FB7F894282F3327AA
:100400008BB391E089278BBB2FBF1F5F675F7F4F47
:100410000894E11CF11C133008F4AACF8FB7F894AC
:10042000082F112781E00E9490000FBFDF91CF912C
:100430001F910F91FF90EF90DF90CF90BF90AF9002
:100440009F908F907F906F900895EF920F931F93DE
:10045000AE2D99E0899FF0011124E050FF4F4083B9
:100460005183628373830483158326833783A1704A
:1004700080858E7F8A2B826080878FB7F894082FC3
:10048000112781E00E9490000FBF1F910F91EF9004
:1004900008950F931F93E0911B01EE23D9F58FB7B9
:1004A000F894682F77278091200190912101A091E5
:1004B0002201B091230120911C0130911D01409136
:1004C0001E0150911F01820F931FA41FB51F6FBF04
:1004D0009C014427552780912C0190912D01A091DA
:1004E0002E01B0912F016FB7F894062F112720939A
:1004F00020013093210140932201509323018093E6
:100500001C0190931D01A0931E01B0931F010E9436
:10051000DA000FBF0E94B200DC01CB01AA27BB2783
:10052000AA27BB27BC01CD010E94A3011F910F91F7
:1005300008958F929F92AF92BF92CF92DF92EF92E7
:10054000FF920F931F93CF93DF930E94B200DC01C1
:10055000CB01AA27BB274C01AA24BB243FEFC32E03
:100560003FEFD32E3FEFE32E3FE7F32E10E087B7A8
:100570008D7F87BF60E071E002E0EB01888581FF3D
:100580001CC088819981AA81BB81A5019401281B87
:10059000390B4A0B5B0BDA01C9012C813D814E817D
:1005A0005F81281B390B4A0B5B0B2C153D054E0553
:1005B0005F051CF469017A0111E00150675F7F4F0C
:1005C00007FFDBCF112361F11C141D041E041F045F
:1005D0002CF0C501B4010E94A30122C0C0922C01DD
:1005E000D0922D01E0922E01F0922F0181E08093B4
:1005F0001B018FB7F894082F112780922001909249
:100600002101A0922201B0922301C0921C01D0923C
:100610001D01E0921E01F0921F010E94DA000FBF3F
:10062000DF91CF911F910F91FF90EF90DF90CF90CE
:10063000BF90AF909F908F900895809130018F3F31
:10064000C9F09091300180913001E82FFF27EF5CD5
:10065000FE4F808180933001809130018F3F11F4F3
:1006600080933301892F9927FC01EF5CFE4F2FEF18
:10067000208302C08FEF90E08F3F19F480E090E07C
:1006800008959927009719F0019721F005C00E945D
:10069000490202C00E94990281E090E008951F92F1
:1006A0000F920FB60F9211248F938FB18091250175
:1006B0008FB98F910F900FBE0F901F901895CFEFAD
:1006C000D0E1DEBFCDBF8FB7F894E82E8FEF9FEF5C
:1006D00090933201809331018FEF809330018093AA
:1006E000330181E08EBD88E080BF83E083BF2CB5FD
:1006F0003DB54AE78CB59DB58217930708F4415084
:100700009C014423B9F792B782B78917E9F32CB556
:100710003DB592B782B78917E9F38CB59DB5821BB9
:10072000930B409645E0969587954A95E1F790930F
:100730002B0180932A0113BE83B78EBD8EB580BF77
:1007400012BE1DBC1CBC8FEF86BF86B780937C0099
:1007500080B7082F11270770107001151105C1F718
:10076000D29AD19AD09ADA9AD99AD89A05BB8FEFB1
:1007700084BBD498DC9880B7886080BFD6988C9A68
:100780008E9A8F9A949A979A969A6FE3802F0E94E6
:100790006E00602F8BE00E946E00B998BF98BB98E6
:1007A000BA9880E285BF0E941D038823E1F700B656
:1007B00002FCFDCF12BE87B7816087BF83B7887FF9
:1007C000836000B600FCFDCF83BF0E941D03C82FCD
:1007D000DD27CC23D1F7EFBE78940E94B200DC0174
:1007E000CB01AA27BB27AA27BB27EC2E09E110E0E3
:1007F00020E030E0AC01BD018C2F0E9425020E9458
:10080000B200DC01CB01AA27BB27AA27BB2702E342
:1008100010E020E030E0AC01BD0181E00E94250243
:100820000E94B200DC01CB01AA27BB27AA27BB2765
:1008300004E610E020E030E0AC01BD0182E00E945F
:1008400025028FB7F894482F4AC087B79927887B2D
:10085000892B41F480917D00282F33272B7F211590
:10086000310519F020E030E02AC06F9928C08AB124
:10087000807C29F580919A00807C09F5379B03C024
:1008800021E030E01CC087B7992783709070892BD6
:10089000A1F080B7992787709070892BD1F781B725
:1008A00092B7891B8C3018F082B7853F18F022E090
:1008B00030E005C023E030E002C025E030E0E5E0B4
:1008C0002E1708F4E22F85B7837EFF27E457FF4FEA
:1008D0009491892B806285BF78948895F894809153
:1008E00030018F3FC9F09091300180913001E82FA5
:1008F000FF27EF5CFE4F80818093300180913001B3
:100900008F3F11F480933301892F9927FC01EF5C0D
:10091000FE4F2FEF208302C08FEF90E08F3F09F44E
:1009200094CF4FBF9927009719F0019721F089CFF5
:100930000E94490286CF0E94990283CF1F920F9294
:100940000FB60F9211240F931F932F933F934F9342
:100950005F936F937F938F939F93AF93BF93CF9347
:10096000EF93FF9383B783BF00B600FCFDCF87B73B
:100970008D7F87BF78948FB7F894C82F80911C0122
:1009800090911D01A0911E01B0911F010097A1053A
:10099000B10549F48FB7F894082F112780E00E9421
:1009A00090000FBF02C00E94DA00CFBFFF91EF910D
:1009B000CF91BF91AF919F918F917F916F915F91F7
:1009C0004F913F912F911F910F910F900FBE0F905C
:1009D0001F9018951F920F920FB60F9211242F930C
:1009E0003F934F935F936F937F938F939F93AF93B7
:1009F000BF93EF93FF9383B783BF00B600FCFDCF97
:100A00008091260190912701A0912801B0912901A0
:100A10000196A11DB11D8093260190932701A093FB
:100A20002801B093290180912401882339F0815055
:100A300080932401882311F40E94DA00FF91EF9142
:100A4000BF91AF919F918F917F916F915F914F91E6
:0E0A50003F912F910F900FBE0F901F901895A1
:00000001FF
